BL51 BANKED LINKER/LOCATER V5.11                                                        02/09/2014  14:36:24  PAGE 1


BL51 BANKED LINKER/LOCATER V5.11, INVOKED BY:
D:\PROGRAM FILES\KEIL\C51\BIN\BL51.EXE STARTUP.obj, 接收文件.obj TO receive_data RAMSIZE (64)


MEMORY MODEL: SMALL


INPUT MODULES INCLUDED:
  STARTUP.obj (?C_STARTUP)
  接收文件.obj (接收文件)


LINK MAP OF MODULE:  receive_data (?C_STARTUP)


            TYPE    BASE      LENGTH    RELOCATION   SEGMENT NAME
            -----------------------------------------------------

            * * * * * * *   D A T A   M E M O R Y   * * * * * * *
            REG     0000H     0008H     ABSOLUTE     "REG BANK 0"
            DATA    0008H     0004H     UNIT         ?DT?接收文件
            IDATA   000CH     0001H     UNIT         ?STACK

            * * * * * * *   C O D E   M E M O R Y   * * * * * * *
            CODE    0000H     0003H     ABSOLUTE     
            CODE    0003H     0012H     UNIT         ?PR?_DELAY?接收文件
            CODE    0015H     0012H     UNIT         ?PR?INIT?接收文件
            CODE    0027H     0010H     UNIT         ?PR?MAIN?接收文件
            CODE    0037H     000CH     UNIT         ?C_C51STARTUP
            CODE    0043H     000BH     UNIT         ?PR?RECEIVE?接收文件



OVERLAY MAP OF MODULE:   receive_data (?C_STARTUP)


SEGMENT
  +--> CALLED SEGMENT
---------------------
?C_C51STARTUP
  +--> ?PR?MAIN?接收文件

?PR?MAIN?接收文件
  +--> ?PR?INIT?接收文件
  +--> ?PR?RECEIVE?接收文件
  +--> ?PR?_DELAY?接收文件



SYMBOL TABLE OF MODULE:  receive_data (?C_STARTUP)

  VALUE           TYPE          NAME
  ----------------------------------

  -------         MODULE        ?C_STARTUP
  C:0037H         SEGMENT       ?C_C51STARTUP
  I:000CH         SEGMENT       ?STACK
  C:0000H         PUBLIC        ?C_STARTUP
BL51 BANKED LINKER/LOCATER V5.11                                                      02/09/2014  14:36:24  PAGE 2


  D:00E0H         SYMBOL        ACC
  D:00F0H         SYMBOL        B
  D:0083H         SYMBOL        DPH
  D:0082H         SYMBOL        DPL
  N:0000H         SYMBOL        IBPSTACK
  N:0100H         SYMBOL        IBPSTACKTOP
  N:0080H         SYMBOL        IDATALEN
  C:003AH         SYMBOL        IDATALOOP
  N:0000H         SYMBOL        PBPSTACK
  N:0000H         SYMBOL        PBPSTACKTOP
  N:0000H         SYMBOL        PDATALEN
  N:0000H         SYMBOL        PDATASTART
  N:0000H         SYMBOL        PPAGE
  N:0000H         SYMBOL        PPAGEENABLE
  D:00A0H         SYMBOL        PPAGE_SFR
  D:0081H         SYMBOL        SP
  C:0037H         SYMBOL        STARTUP1
  N:0000H         SYMBOL        XBPSTACK
  N:0000H         SYMBOL        XBPSTACKTOP
  N:0000H         SYMBOL        XDATALEN
  N:0000H         SYMBOL        XDATASTART
  C:0000H         LINE#         92
  C:0037H         LINE#         99
  C:0039H         LINE#         100
  C:003AH         LINE#         101
  C:003BH         LINE#         102
  C:003DH         LINE#         151
  C:0040H         LINE#         155
  -------         ENDMOD        ?C_STARTUP

  -------         MODULE        接收文件
  C:0000H         SYMBOL        _ICE_DUMMY_
  D:0090H         PUBLIC        P1
  D:00A0H         PUBLIC        P2
  B:0098H.0       PUBLIC        RI
  D:0008H         PUBLIC        flag
  D:0009H         PUBLIC        Receive_Data
  C:0027H         PUBLIC        main
  D:0099H         PUBLIC        SBUF
  D:0087H         PUBLIC        PCON
  D:0098H         PUBLIC        SCON
  D:0089H         PUBLIC        TMOD
  C:0015H         PUBLIC        init
  D:000AH         PUBLIC        flag1
  D:008DH         PUBLIC        TH1
  D:008BH         PUBLIC        TL1
  D:000BH         PUBLIC        pf
  B:0088H.6       PUBLIC        TR1
  C:0043H         PUBLIC        receive
  C:0003H         PUBLIC        _delay
  B:00A0H.0       PUBLIC        key2
  -------         PROC          _DELAY
  D:0007H         SYMBOL        k
  -------         DO            
  D:0006H         SYMBOL        j
  -------         ENDDO         
  C:0003H         LINE#         26
BL51 BANKED LINKER/LOCATER V5.11                                                      02/09/2014  14:36:24  PAGE 3


  C:0003H         LINE#         27
  C:0003H         LINE#         29
  C:0009H         LINE#         30
  C:0009H         LINE#         31
  C:0011H         LINE#         32
  C:0014H         LINE#         33
  C:0014H         LINE#         34
  -------         ENDPROC       _DELAY
  -------         PROC          INIT
  C:0015H         LINE#         45
  C:0015H         LINE#         46
  C:0015H         LINE#         47
  C:0018H         LINE#         48
  C:001BH         LINE#         49
  C:001EH         LINE#         50
  C:0021H         LINE#         51
  C:0023H         LINE#         52
  C:0026H         LINE#         53
  -------         ENDPROC       INIT
  -------         PROC          RECEIVE
  C:0043H         LINE#         64
  C:0043H         LINE#         65
  C:0043H         LINE#         66
  C:0045H         LINE#         67
  C:0047H         LINE#         68
  C:004AH         LINE#         69
  C:004AH         LINE#         71
  C:004AH         LINE#         72
  C:004DH         LINE#         73
  -------         ENDPROC       RECEIVE
  -------         PROC          MAIN
  C:0027H         LINE#         84
  C:0027H         LINE#         85
  C:0027H         LINE#         86
  C:002AH         LINE#         87
  C:002AH         LINE#         88
  C:002AH         LINE#         89
  C:002DH         LINE#         90
  C:0032H         LINE#         91
  C:0035H         LINE#         92
  -------         ENDPROC       MAIN
  -------         ENDMOD        接收文件

Program Size: data=13.0 xdata=0 code=78
LINK/LOCATE RUN COMPLETE.  0 WARNING(S),  0 ERROR(S)
